:10000000A7C0C0C0BFC0BEC0FFC0BCC0BBC0BAC0DC
:10001000B9C00AC2B7C044C6B5C0B4C0B3C0B2C04C
:1000200019C1B0C0AFC09AC7BDC7D3C794C704C871
:1000300017C82BC8CEC7CDC752C866C86DC8CCC7B5
:1000400092C8B0C788C721C84AC84552523A204210
:10005000756666657220456E6420726561636865C9
:10006000640D0A0056312E30623136004150525331
:10007000206E616E6F2D544E4320006563686F00E3
:1000800000000000006D7963616C6C00000000638B
:100090006F6E76657273650000747864656C617963
:1000A00000000063616C00000000000000746F6ECF
:1000B00065000000000000756E70726F746F0000C4
:1000C000006B000000000000000000636F6E76000F
:1000D00000000000006465627567000000000072A7
:1000E00065737461727400000073746F7265000050
:1000F00000000074787461696C000000006B697323
:10010000730000000000006D790000000000000096
:100110000074786400000000000000756E7000003C
:100120000000000000646562000000000000003F65
:100130004548002E2E2E0053594E5441580D0A00AA
:10014000206F666600206F6E00636D643A200000C9
:1001500011241FBECFE5D4E0DEBFCDBF10E0A0E686
:10016000B0E0E2EEF3E102C005900D92AA37B107CC
:10017000D9F713E0AAE7B0E001C01D92A435B1079A
:10018000E1F7FAC23DCF10928C002091B40130917A
:10019000B50191E0E8E0F4E8482F55274170507030
:1001A000B901642775273695279560FF02C02E2771
:1001B0003F279F5F993011F08695EECF88E08093BE
:1001C0008C0070938900609388003093B501209370
:1001D000B40150938B0040938A00089591E090936E
:1001E0005303A895809582BF809153038823E1F73C
:1001F000089591E090930003A895809584BD809127
:1002000000038823E1F708951F920F920FB60F9213
:1002100011248F93EF93FF938091B201882379F09B
:10022000E0917D00EF5FEF70E0937D00FF27E05AE3
:10023000FF4F808185BB8091FF0284BD03C0109277
:10024000000314BCFF91EF918F910F900FBE0F90A0
:100250001F9018951F920F920FB60F9211242F9393
:100260003F938F939F939D9B02C0AD9801C0AD9A21
:100270008091B0019091B101892B09F03FC02CB55C
:100280003DB530937C0020937B0082E02F3138070E
:10029000B0F01DBC1CBC80917A00803D39F481E037
:1002A0008093B3013093B7012093B60184EA809321
:1002B0007A008091FD02823009F58DE41EC0293C50
:1002C0003105B0F01DBC1CBC80917A00843A39F431
:1002D00081E08093B3013093B7012093B60180EDA4
:1002E00080937A008091FD02823041F483E505C05D
:1002F0008091FD02882311F088E48CB99F918F9141
:100300003F912F910F900FBE0F901F9018951F9344
:10031000182F16951F7051F08DE2A1D41A3018F0E5
:1003200081E39DD41A50812F805D99D41F91089547
:10033000CF92DF92EF92FF920F931F93CF93DF93B1
:10034000CDB7DEB721970FB6F894DEBF0FBECDBF95
:100350007C018C01DD24F8018781803441F0869591
:100360007ED4D3940F5F1F4FF6E0DF16A1F7F7019D
:100370008585CDDFF7018585817089838EE36FD414
:10038000870186E0C82ED12CCE0CDF1CF8018191AC
:100390008F01803429F0869562D40C151D05B1F7C4
:1003A000F7018681B4DF8981882379F58EE090E0BA
:1003B000E80EF91E8CE253D425C08701B6E0CB2E9F
:1003C000D12CCE0CDF1CF80181918F01803429F0F3
:1003D000869545D40C151D05B1F7F7018681982F38
:1003E0009170998394DFF701868187FF02C08AE2CA
:1003F00036D48981882311F48CE231D487E090E0EF
:10040000E80EF91E89818130C1F621960FB6F89465
:10041000DEBF0FBECDBFDF91CF911F910F91FF9037
:10042000EF90DF90CF9008951F920F920FB60F922A
:1004300011241F932F933F934F935F936F937F9359
:100440008F939F93AF93BF93CF93DF93EF93FF93DC
:100450008091B201882321F01092530312BE5CC137
:1004600085E482BF8091B6019091B701009709F4AD
:1004700045C101979093B7018093B6018091F20234
:10048000882309F4C09A81E08093F2028091B3013D
:10049000882341F1809183008530D1F0AC98809120
:1004A00084008F5F8093840080918500869580937F
:1004B00085008091FD02833010F080E3D0D38091DD
:1004C0008300863029F480917E00826080937E00D4
:1004D0001092B30110928300109287008CE08093F9
:1004E000860039C0809187008F5F8093870090914C
:1004F00086008917E1F4AC9A809183008F5F809326
:100500008300809184008F5F8093840080918500B8
:1005100086958068809385001092870088E080939C
:1005200086008091FD02833010F081E398D38091A2
:1005300083008F3080F0109283001092B7011092E8
:10054000B6018091FD02882331F08FE388D380913A
:10055000FD0281119CD320917E0021FF21C080915A
:1005600085008E37E9F48FEF9FEF9093B50180936C
:10057000B4011092840010928100109280001092B9
:10058000820010927F0021602D7F20937E00809159
:10059000FD02882311F08AE362D310928500BCC06B
:1005A00020FFBAC080918400883009F0B5C08091E6
:1005B000FD02882311F081E252D3709182007723EB
:1005C00009F459C0609185004091B4015091B50182
:1005D000262F3327842F809599272817390751F51F
:1005E000852F9927809580937F008091FD02882335
:1005F00009F441C084E433D38091FD028430D8F102
:1006000088E22DD3C0E0D0E080917F0099270C2EA6
:1006100002C0959587950A94E2F780FF02C081E3B6
:1006200001C080E31CD32196C830D10569F789E267
:1006300016D321C080917F008823D9F06817C9F4B0
:100640007093AF01E0918000F09181003297F093B8
:10065000B101E093B001E157FF4F118280917E001C
:100660008E7F80937E008091FD02882321F00FD33E
:1006700002C010927F0010918500812F84DD80914F
:10068000B0019091B101892BE1F4809180009091AB
:100690008100FC01E157FF4F108301969093810088
:1006A000809380008052914061F480917E008E7F23
:1006B00080937E008091FD02882319F08AE490E007
:1006C000D2D2209180003091810025FE07C02E30CB
:1006D000310589F48EE0809382000DC0F901E15765
:1006E000FF4F82913196803F31F432978081833081
:1006F00011F420938200109284000EC08091F202C7
:10070000882351F01092F202C098109284008091D8
:100710007E008E7F80937E00FF91EF91DF91CF91DD
:10072000BF91AF919F918F917F916F915F914F9109
:100730003F912F911F910F900FBE0F901F90189512
:10074000E1D11092B201C19882E083BF8EBD87E0F3
:1007500085BD439A579A0895439883E083BF82E00A
:100760008EBD85BD81E08093B201C19A822D8871D2
:1007700011F45798ECD10895CFE5D4E0DEBFCDBF9A
:1007800060D215BA84B38F6384BB18BA87B3836011
:1007900087BB80EE87B910BE88E088B982E083BF4E
:1007A0008EBD17E015BD81E489BF88E190E02EE0A1
:1007B0000FB6F894A89581BD0FBE21BD84EE282206
:1007C00084E0282A8FED2822F2D48091F1028F3F15
:1007D00019F48CE18093F1028091FE028F3F11F4B5
:1007E0001093FE027894A89510928E0010928D00BE
:1007F000C0E0D0E08AEFFDDC2196CA30D105D1F708
:100800008AE090E090938E0080938D008CE690E0DB
:100810002AD284E690E027D23AD239D236D3822D3A
:1008200020FE1BC0827281F08091F202882321F0A9
:100830008091B601DEDCF3CF8EEF28228DDF86ECCF
:1008400091E02AD17DDFEBCF8091C601882311F49E
:100850001CD301C033D38EEF28228091B001909138
:10086000B101892BE9F125FE2BC080ECF8D180E0A5
:10087000F6D110928E0010928D00E0E0F0E0E1578A
:10088000FF4F8081803C21F48BEDE9D18CED04C0D9
:100890008B3D11F4E4D18DEDE2D1E0918D00F0912A
:1008A0008E003196F0938E00E0938D008091B00120
:1008B0009091B1018E179F0710F780ECD0D10CC03A
:1008C0008FE890E035DD8AE3CAD18091AF019927A6
:1008D00081579F4FD2D1DBD11092B1011092B0015C
:1008E00023FE08C039DF03C080E02DD0A89523FC8B
:1008F000FBCF26DF24FE0AC084EA8093FF022CDFB0
:1009000002C08AEF6BDC24FCFCCF1ADFA89587CFEE
:100910002091C2013091C301822793279093BA019D
:100920008093B901369527953093C3012093C20176
:1009300080FF08C088E094E8282739273093C30156
:100940002093C20108951F93CF93DF93182F8093B4
:10095000BE011092BF018091BE01C82FDD27C7FDE7
:10096000D095C170D070D093BD01C093BC011E372B
:1009700019F41092BB0102C0CE01CADFCD2B61F485
:100980001092BB018091FF02843A11F480ED01C006
:1009900084EA8093FF0214C08091BB018F5F809333
:1009A000BB01853069F48DEB19DC8091FF02843A3C
:1009B00011F480ED01C084EA8093FF021092BB0124
:1009C0008091BE0185958093BE018DEB07DC8091FF
:1009D000BF018F5F8093BF0188300CF4BCCFDF91E3
:1009E000CF911F910895DF92EF92FF920F931F9383
:1009F000CF93DF93CDB7DEB722970FB6F894DEBF63
:100A00000FBECDBF8C016A8319826DE270E044D4C1
:100A10007C010894E11CF11CDD24F80190819D32D9
:100A200039F0992329F0903219F08981882321F037
:100A300081E0898380E402C0892F880F84DFD3940A
:100A4000F6E0DF1619F00F5F1F4FE7CF81E0E816E1
:100A5000F10411F420E009C0F701208120538181C5
:100A6000882311F0280F2752220F922F90668A8137
:100A7000882311F0922F9166892F65DF22960FB699
:100A8000F894DEBF0FBECDBFDF91CF911F910F91C4
:100A9000FF90EF90DF900895CF93DF93EC0102C0B9
:100AA00052DF219688818823D9F7DF91CF9108956D
:100AB000CF93DF93EC01885E934010F0C7EED3E054
:100AC0001092B80180E003C0C456D0408F5FC43696
:100AD000D105D0F78093B801805D35DF1092B80161
:100AE00080E002C02A978F5FCA30D105D8F7809383
:100AF000B801805D28DF9E01205D822F24DFDF9119
:100B0000CF910895CF93DF938091C2019091C3015B
:100B1000292F332720952093C001809514DF8091E1
:100B2000C00111DFC0E0D0E003C08EE70CDF2196EA
:100B30009091FE028AE0989FC001112467E070E066
:100B4000F8D3C617D7078CF3DF91CF9108950F9391
:100B50001F93CF93DF93CDB7DEB72A970FB6F894E4
:100B6000DEBF0FBECDBF8FEF9FEF9093C301809389
:100B7000C2011092C10107C08EE7E5DE8091C1017C
:100B80008F5F8093C1012091C10133279091F102C1
:100B90008AE0989FC001112467E070E0CAD326174D
:100BA000370754F325FC42C060E087EE92E01BDF7C
:100BB00080910303882391F160E083EF92E013DFDB
:100BC00003E013E025C06CE270E0C80165D3892B17
:100BD00011F120E030E0CE01019603C0A80FB91F4B
:100BE000EC93A22FBB27F801EA0FFB1FE0812F5FD8
:100BF0003F4FEC3299F7A80FB91FFD01118260E059
:100C0000F2DE6CE270E0C80147D38C010F5F1F4F2A
:100C100001301105C1F661E0C80103C061E083EF56
:100C200092E0E1DE83E08FDE80EF8DDE2A960FB664
:100C3000F894DEBF0FBECDBFDF91CF911F910F9112
:100C400008958898909A8FE089B910BC86E880BD95
:100C500088E98AB9109202031092010308955D9BFE
:100C6000FECF8CB90895FC0104C05D9BFECF319688
:100C70008CB984918823C9F70895FC0104C05D9B59
:100C8000FECF31968CB980818823C9F708955D9B8A
:100C9000FECF8DE08CB95D9BFECF8AE08CB90895C4
:100CA0001F920F920FB60F9211241F932F933F9311
:100CB0004F935F936F937F938F939F93AF93BF9364
:100CC000EF93FF931CB18091010390910203815235
:100CD000914021F41092020310920103822D25FE0F
:100CE0006CC08091C50181FF61C08091C50182FD0A
:100CF00008C0112311F01093C4018091C5018460D4
:100D000044C08091C401882389F0843039F08F3F3A
:100D100041F0813041F41093F10205C01093FE02BE
:100D200002C08FED28221092C40194C0103CB9F487
:100D3000E0910103F0910203309731F021E0222A83
:100D40005798EA53FE4F10828091C5018D7F8093A2
:100D5000C5018091C5018B7F8093C50133C080910F
:100D6000C50180FF0DC01C3D11F410EC03C01D3DFA
:100D700009F41BED8091C5018E7F8093C50108C0E9
:100D80001B3D31F48091C50181608093C50162C033
:100D90008091010390910203FC01EA53FE4F1083FE
:100DA0000196909302038093010354C0103C09F014
:100DB00051C08091C5018260E8CF133041F465D005
:100DC00085EE2822109202031092010343C024FEF4
:100DD0000CC0103251F48091FF02843A11F480ED7E
:100DE00001C084EA8093FF0235C01D3099F482FD72
:100DF0004EDFE0910103F0910203EA53FE4F1082AF
:100E0000109202031092010321E0222A21FE1DC04C
:100E100057981BC08091010390910203183061F430
:100E20000097C1F0019790930203809301035D9BAB
:100E3000FECF88E08CB90EC0FC01EA53FE4F108350
:100E40000196909302038093010322FE03C05D9BF1
:100E5000FECF1CB9FF91EF91BF91AF919F918F9100
:100E60007F916F915F914F913F912F911F910F90C3
:100E70000FBE0F901F901895892B19F085E491E013
:100E800002C080E491E0EFDE089589E491E0EBDEBA
:100E900008950F931F93CF93DF938C01EC0105C04E
:100EA000992787FD90956CD2899388818823C1F713
:100EB000C801DF91CF911F910F910895DF92EF92BA
:100EC000FF920F931F93CF93DF93CDB7DEB7629757
:100ED0000FB6F894DEBF0FBECDBF86EC91E09A83CB
:100EE000898380E1FE01339611928A95E9F7FF2408
:100EF00060E770E08E010F5F1F4FC801E8D1DC0191
:100F0000EF2DFF27EE0FFF1FE00FF11FB383A2832A
:100F1000109731F08C918111F39428E02F1540F750
:100F2000EB80FC80DD240BE710E0B801C7018FD116
:100F3000892B49F4ED2DFF27E231F10508F024C19A
:100F4000ED5EFF4F0994D394065F1F4F85EBD816D3
:100F500009F41AC1EACF01EF12E040C00D811E81F1
:100F600001151105A9F062E770E0C80183D1892B52
:100F700019F494E0292A0CC065E770E0C8017AD121
:100F8000892B19F4ABEF2A2203C087E391E06BDED3
:100F90008BE790E068DE822D869586958170992793
:100FA0006BDFF5C08AE0D89EC001112485589F4FA1
:100FB0005ADE80E254DE8D819E81009739F069DF30
:100FC0004AE050E0BC0183EF92E072D183EF92E0FF
:100FD00084C0B2E02B2ADDC00EEF12E08D819E812D
:100FE000009741F008D18F3F910511F008F0CCC077
:100FF000F80180838AE0D89EC001112485589F4F54
:1010000032DE80E22CDED8018C9164E686D1882322
:1010100011F0805D24DEF801808164E67ED1892FA5
:101020006AE07BD1882311F0805D19DED8018C91B4
:101030006AE073D1892F65C0822D86958695869545
:1010400080958170880F880F880FB7EF2B22282A90
:1010500083EA90E008DE822D86958695869510C0FD
:10106000822D82958F70809581708295807FEFEEC2
:101070002E22282A8DEA90E0F6DD822D82958F704F
:1010800081709927F9DE03DE84C08AE0D89EC00112
:10109000112485589F4FE7DD80E2E1DD8D819E813F
:1010A0000097A1F0F6DE4AE050E0BC0187EE92E046
:1010B000FFD01092030389859A85009739F0E9DE05
:1010C00040E550E0BC0183E093E0F2D087EE92E08F
:1010D000D4DD80E2C4DD83E093E0CFDD58C08D81B4
:1010E0009E81009719F087D08093FD028AE0D89EF8
:1010F000C001112485589F4FB6DD80E2B0DD80919C
:10110000FD02805DACDD43C08FED90E0ACDD83E39C
:1011100091E0A9DDBCDDFFCF89EE90E0A4DD8AE09F
:10112000E3EFF2E040E050E0DA01182E48D1E7EEBC
:10113000F2E0465F5F4FDA01182E41D180E5E3E02F
:10114000F3E0465F5F4FDA01182E39D18091F1024A
:10115000A4E6B0E0082E27D18091FE02A5E6B0E01B
:10116000082E21D114C08DEF90E07DDD822D829577
:101170008695877080958170982F9295990F907EB3
:10118000BFED2B22292A7DCF8FE291E06CDD7FDD40
:101190007CDE62960FB6F894DEBF0FBECDBFDF9146
:1011A000CF911F910F91FF90EF90DF9008958AE00B
:1011B000E3EFF2E040E050E0DA01182EEFD0E7EE86
:1011C000F2E0465F5F4FDA01182EE8D080E5E3E0F9
:1011D000F3E0465F5F4FDA01182EE0D0A4E6B0E0FE
:1011E000D5D0802D8093F102A5E6B0E0CFD0802D40
:1011F0008093FE020895FC0188279927E8942191A5
:101200002223E9F02032D9F32930C9F32A30B9F387
:101210002C30A9F32D3099F3263789F32B3219F0AE
:101220002D3221F468942191222349F020333CF09F
:101230002A332CF4205369D0820F911DF4CF8115ED
:10124000910521F01EF48095909501960895FB017B
:10125000DC018D910590602D502D5062513624F0A7
:101260005B3714F460628062861B11F4002089F7FA
:10127000990B0895FB01DC018D916191562F50620D
:10128000513624F05B3714F460628062861B11F4DF
:10129000662391F7990B0895FC010190061629F039
:1012A0000020D9F78827992708953197CF0108950D
:1012B000FB01DC014150504048F001900D920020AC
:1012C000C9F701C01D9241505040E0F70895DC017C
:1012D0004D915C914115510519F48827992708957E
:1012E000DA013D91FB012191231761F4332319F4B5
:1012F000AA27BB2702C01E921196FC01A193B083BE
:10130000CA010895222379F7ECCF7AE0979F902DB8
:10131000879F802D910D11240895991B79E004C0B9
:10132000991F961708F0961B881F7A95C9F7809524
:10133000089597FB092E07260AD077FD04D00CD01C
:1013400006D000201AF4709561957F4F0895F6F746
:10135000909581959F4F0895AA1BBB1B51E107C033
:10136000AA1FBB1FA617B70710F0A61BB70B881F35
:10137000991F5A95A9F780959095BC01CD010895C4
:101380008F9324D08F9109F08F7D0895E199FECF3E
:10139000BFBBAEBBE09A11960DB20895F7DF019284
:1013A0001A94E1F70895E199FECFBFBBAEBB0DBA29
:1013B00011960FB6F894E29AE19A0FBE0895019043
:1013C000F2DF1A94E1F7089585FD08C0806291115B
:1013D00005C08136ECF38B37DCF708959927882711
:0213E00008956E
:1013E200070A0D0E0F0E0D0A080502010001020583
:0A13F20020006F6E006F66660000B9
:00000001FF
